:1000000000308A0089290000663084000008031946
:1000100019280130F800BF30F7006400F70B0D28F5
:10002000F80B0B284230F700F70B14286400800B04
:1000300009280034831605178312051F212805138C
:10004000222805178316051383128A11292AE6012F
:100050006608F93C031C4728651830280513312829
:1000600005178316051301308312E50665183A2833
:1000700085133B2885178316851364001F30F7000E
:10008000F70B4028000000008312E60A2828831698
:1000900005138312051783168513831285178A119A
:1000A000762A5F08840067088000840A8001DF0ADE
:1000B00000346808F8016702031861286708F70030
:1000C0006D28F7010830E900E70DF70D68087702A1
:1000D0000318F700F80DE90B642800347808650868
:1000E000E7006430E80059207708E50078083030F0
:1000F000031D8128E61C8828E6198828661A203006
:100100008428E61166126614F8077808E700512083
:100110006508E7000A30E80059207708E50078080C
:100120003030031D9928E6199D28661C9D28661A03
:100130002030F8077808E70051203030E5076508DF
:10014000E70051200034B301301CA8283010A92842
:1001500030140034301CD62883168612831286127F
:1001600064004730F700F70BB328000083168612AF
:100170008312861664004730F700F70BBD28000095
:10018000831686128312861264004730F700F70B3D
:10019000C728000083168612831286166400183062
:1001A000F700F70BD12800000000E928831686121B
:1001B0008312861264008530F700F70BDD28831662
:1001C00086128312861664006F30F700F70BE6285C
:1001D00000000034E8016808073C031C3229670866
:1001E0000139E900B5080319F7280030F828013073
:1001F000EA00B4080319FE280030FF2801306A0520
:10020000003A031912296908EA000310B20CB10C74
:10021000030801396A06013C031D12298430B20625
:100220000830B106E908031D1729A3202D29B408B9
:100230000319B30AB40803191F290030202901301B
:10024000EA003308053C031927290030282901302A
:100250006A0503192D29AA20A320AA200310E70C60
:10026000E80AEB2800343010FF30B200B100B301CF
:100270000130B400B501B6013608093C031C45291C
:100280007E30E700EA20B60A3C29B401B601360800
:100290000F3C031C54292030360784000008E60078
:1002A000E700EA20B60A4729B6016508840000087D
:1002B00003196329650884000008E600E700EA20C6
:1002C000E50AB60A55290130B500FF30B106B2067D
:1002D0003108E700EA203208E700EA20B5010130E2
:1002E000B4007E30E700EA208A11C22A1230E6020A
:1002F000031C882966308400FC3080050310800CC4
:10030000800C00080319882986296400800B852940
:10031000003484011F30830583161F129F121B08AF
:1003200080399B0007309C0082308312A0009830F7
:10033000A100A2004030A300A400A5006030A600E8
:100340008630A700B430A8006030A900A430AA000D
:10035000AB00AC006130AD000330AE00F030AF0058
:10036000DF0183160108C03981000E30F700073025
:1003700083128101813084000008F0390738800041
:1003800064000008F739F719F0397704800090010C
:1003900083161F129F121B088039D3389B001F132E
:1003A00083121F179F1783169F1383121F14941213
:1003B00083160611861406120030831294008316E9
:1003C000940007309C00050864000230F700F70B2A
:1003D000E72900001C0883120D1383169D01861166
:1003E0008312861183160611831206118316861056
:1003F00083128610831685138312851783160513BF
:10040000831205172030F8001F08C73978049F00B1
:10041000950183168611831286110C3097000030E7
:10042000F8000438920064308316920062308F0026
:10043000023083129500E001831686108312861025
:100440006430E60004206008E00A043C031D2A2A08
:100450001A28E00183168610831286140130E60004
:1004600004201F151F19322A1E085F3C031C1C2A7A
:1004700083168610831286100030F8001F08C739D3
:1004800078049F0064001F30F700F70B452A000036
:1004900000001F151F194A2A1E08F700F70CF70C59
:1004A0003F30F7057708283EE1000830F8001F08C4
:1004B000C73978049F0064001F30F700F70B5E2AED
:1004C000000000001F151F19632A1E081E0EE200FF
:1004D0000F30E20595010030F80004389200610801
:1004E0008316920013308312950027280230E5000E
:1004F000FA30E6000420E50B782A83168610831272
:1005000086142030F8001F08C73978049F00640063
:100510000F30F700F70B8A2A00001F151F198E2ACB
:100520001E08E30083168610831286103730DF0022
:100530007030E70051203D30E70051206108E500B0
:100540001B30E6006E202030E70051207230E700BB
:1005500051203D30E70051206208E5001B30E600E5
:100560006E202030E70051207530E70051203D30EB
:10057000E70051206308E5001B30E6006E203730AD
:10058000E50033293830E500FA30E6000420E50BB9
:10059000C42A0130E400640FCE2AEF2AE00160088B
:1005A0006202031CED2A83160611831206156408E5
:1005B000E60076216408E600762183160611831290
:1005C00006116408FF3CE500E60076216408FF3C64
:1005D000E500E6007621E00ACF2AE40ACB2A83165A
:1005E0000611831206150A30E5008230E600042069
:1005F000E50BF52A83160611831206118A010028DD
:02060000630095
:04400E003827FC3F14
:00000001FF
